:100000008301850186012028A0000308A100830147
:100010000B1D1628A90B1628E130A900AA0B1628DB
:100020003C30AA00AB0B162885118B120B1121084E
:1000300083002008090082077F34BF349334D3340F
:1000400003138316F03085000630860005309900D2
:1000500026309800823081000313831207309F00FE
:1000600020309500043092003C309700903098008A
:1000700020308B00203084008001840A841F3C28BB
:100080009630A6005021A60B422806168616682137
:100090002930A6005021A60B4A286821502168214A
:1000A000061268212830A30059210D30A3005921E0
:1000B0000130A30059210630A30059212B30A300A1
:1000C000592185158B174B21FE3C031969285521B1
:1000D00063284B212308233C03194A292308373C72
:1000E0000319F22823083D3C03194A292308423CFE
:1000F0000319F5282308433C03192D292308443C00
:1001000003192F292308463C031904292308473CD7
:10011000031923292308483C0319D72823084A3CFC
:100120000319152923084B3C03191C2923084C3CAF
:1001300003194A2923084D3C03194A2923084E3C38
:10014000031935292308503C0319E5282308513C9D
:10015000031931292308523C031933292308533C3E
:10016000031907292308543C03190E292308563C78
:100170000319DF282308573C0319E2282308583CB9
:100180000319DB282308683C03194A2923086E3C1D
:1001900003194A292308733C03194A292308763C8A
:1001A00003194A2923087C3C03194A296328033090
:1001B000A300592163280130A300592163284B2152
:1001C000051163284B21051563284B21A30917123C
:1001D000231817169712A3189716A30C230C3F3950
:1001E000950063280530990063288B124B21230862
:1001F00003190229AB003C30AA00E130A9008101BB
:100200000B118B168515632885118B1263280D3011
:10021000221B0238A213A300592163280C30221B91
:100220000238A217A300592163280E30A21F0138FB
:100230002217A300592163280C30A21F0138221372
:10024000A300592163284B21A7004B212303033925
:100250001B202707A30059216328A2166328A21296
:10026000632822166328221263286B212408A70022
:100270004B21A30DA30D230D38394038A30059217C
:100280000830A8004B215521A80B42292708A300BC
:100290005921632863288C1E4B291A08A3000800E3
:1002A0000E30A500A50B522908006B2185100614FD
:1002B0005C296B21851006100F3086052308F03964
:1002C0008604051405100F308605230EF0398604C8
:1002D00005140510080003138316F0308604031379
:1002E000831285140610051406080510F039A400C1
:1002F0000514060E05100F39A404A41B732903135B
:0C03000083160F308605031383120800DB
:02400E00413F30
:00000001FF
